:020000040800F2
:10500000901A0020D55000081D8A00081D81000854
:105010000000000000000000000000000000000090
:105020000000000000000000000000007D96000865
:105030000000000000000000798F0008959700082C
:10504000E7500008E7500008E7500008E750000864
:10505000E7500008C15B0008E7500008E75000086F
:1050600000000000E7500008E95A0008E750000877
:10507000E75000080D86000800000000E750000817
:1050800000000000E75000080000000000000000E1
:10509000E750000800000000E7500008E750000853
:1050A000E7500008E7500008E7500008EDA10008AD
:1050B000E7500008E7500008000000000000000072
:1050C0000348854600F080FC0048004721B80008EE
:1050D000901A00200448804704480047FEE7FEE796
:1050E000FEE7FEE7FEE7FEE731980008C150000842
:1050F00030B50B46014600202022012409E00D4670
:10510000D5409D4205D31D469540491B25469540F7
:1051100040191546521E002DF1DC30BDF0B51FB40C
:105120000646002082B005464024019100901BE015
:10513000019922460F46304600F062FB049A059B17
:10514000801A994110D310461946224600F048FBB8
:10515000361A8F410197224601200021009F00F05E
:105160003FFB38184D4100902046641E0028DFDCCC
:10517000019B00982946324607B0F0BD03460B4319
:105180009B0703D009E008C9121F08C0042AFAD2FD
:1051900003E00B780370401C491C521EF9D2704783
:1051A000D2B201E00270401C491EFBD270470022BF
:1051B000F6E710B513460A4604461946FFF7F0FF16
:1051C000204610BD30B504460020034600E05B1CBD
:1051D000934203D2E05CCD5C401BF8D030BDF8B503
:1051E00002464A40D40F42004B0052085B089A42E4
:1051F00002D20246084611464A0023D0C30D4A0097
:10520000DDB2120EAD1A202D35DA49020126490A07
:10521000F6058A19002C00D0524220214F1B11465E
:10522000B9402A411018C20D9A4221D0002C17D043
:10523000012D08DCDA05801AD20F8019D207DBB203
:1052400000F00AFBF8BDDA05801A012340001B06B6
:10525000C01880185A428018CA0F1043490007E04E
:105260004908C2071143DA05801A801940088018DE
:1052700000F0EAFAF8BD61000122511A001BF7E7BD
:105280000122D2075140AAE70122D2075040A6E7E7
:1052900070B502464A40D50F40004A00ED0740086D
:1052A0005208002814D0002A12D0C40DD30D410298
:1052B0000120C0055202490A520AE41A09181218BC
:1052C0007D34914201D3641C00E04900002C01DAD6
:1052D000002070BD0023914201D3891A0343400886
:1052E00049000028F7D100290AD0914202D10121BA
:1052F000C90705E0914201D2012101E00121C94322
:10530000E005C018401900F09FFA70BDF0B50746DF
:105310000846584087B0C00F049048000E46590018
:1053200040084908BC1A884105D2384631461E4615
:1053300017460B4602465800400810434CD0300D2B
:10534000039040055900400D490D0590401A029008
:10535000402872DA18030121000B09050843019067
:1053600004980092002805D00199524200208841FB
:1053700000920190029840210A1A0199009800F0C9
:105380002FFA05460C466B4607CB00F04AFAC019C7
:105390007141039A0E0D0023D71756401A467A40E2
:1053A000164344D0049A002A2DD0029A012A039A67
:1053B00015DC1205C01A914101263605001C714109
:1053C000D20F059ED2070093019202962A462346E9
:1053D00000F088FA07B0F0BD38463146FAE7160506
:1053E000224A0F46B218C01AB74101210905001C14
:1053F0004F4100187F41114618187941E20F1043C0
:105400006D19644113E0E2076D0815436408C20793
:105410001443039A01261205C01A91413605001C57
:105420007141CE07400830434908C01851412A460F
:10543000234600F04AFACDE7FFE704980122400036
:10544000C117121A00238B4104983146C417381A29
:10545000A141EEE730B40124E407634030BC55E7D6
:1054600030B40124E407614030BC4FE70000E0FFA6
:10547000F0B51FB488B00B990998002448400999E9
:10548000C00F490049080991C0070B9900904900D5
:1054900049080B9109990898A64608431CD00B9916
:1054A0000A98084318D0099801244000420D48008A
:1054B000410D099824050003000B204309900B9827
:1054C0000003000B20430B9050181C494018002289
:1054D00001901446104605E0002001460DB0F0BDD5
:1054E000032801DA034600E003239C46C11A0AAEF2
:1054F0000AE05F0008ADED5B4F00F75B7D430027DE
:10550000AA187C41491C5B1E6145F2DD410004ABD9
:105510005A522104120C0A43240C401C0828DFDBD9
:10552000019802900099704601910090059B049AA1
:105530000799069800F0D6F9D0E700000DFCFFFFB0
:10554000F0B50C465C4085B0E40FE40703944C00D2
:1055500000266408590094464908024602962243F0
:1055600021D062460A431ED06200570D4A000E0346
:105570002303550D012402462C492405781B1B0BDF
:10558000360B401823432643614600901C46501AB0
:10559000B44103D30098401C009002E09218009898
:1055A0005B41002803DA0020014605B0F0BD002071
:1055B000012109050746864611E064461D46141B75
:1055C000B54106D36546521BB341744607430C43AD
:1055D000A646CD0740084908284392185B41054676
:1055E0000D43EAD11046184313D060461946504087
:1055F0007140084306D06046101AB34106D201221A
:10560000002306E000220123DB0702E00122D2434F
:105610005310009874460105381C6141029C039D9B
:105620000019694100F051F9BFE70000FD030000D7
:10563000C217C10F504010B54018CA079623002169
:1056400000F00AF910BD10B500229623114600F0B3
:1056500003F910BD0EB5C217C10F5040CA0740185C
:105660000021054B0293019200910A460B4600F07F
:1056700039F903B000BD0000330400000EB5054940
:105680000291002100910A460B46019100F02AF98F
:1056900003B000BD33040000410040020122400A73
:1056A000D205090E80187F2901DA0020704796295B
:1056B00003DC9622511AC8407047963988407047DB
:1056C00070B5CD0F4A0009030123090B1B051943CF
:1056D0000B4BED070024520D9A4201DA002070BDF9
:1056E000074B34339A4203DC9A1A00F089F802E03F
:1056F0000449511888402C43F1D0404270BD00004D
:10570000FF030000CDFBFFFF4A0009030123090B43
:105710001B051943094B10B5520D9A4201DA0020BE
:1057200010BD064B34339A4203DC9A1A00F068F835
:1057300010BD03495118884010BD0000FF03000050
:10574000CDFBFFFFC20FD207400040080BD0C10DB8
:105750000723DB01C91840020905400A1143C208AA
:1057600040071143704700200146704710B50029DB
:1057700004DB0124E40740428C412146002B04DB7A
:105780001C460123DB075242A341994200D19042BB
:1057900010BD0000CB0FDB07490010B549080246D9
:1057A0000A4307D00A0D07240903E401090B121B61
:1057B000002A01DC002010BDC900440F0C43C100C9
:1057C000E018D205801800F03FF810BD0122D20782
:1057D000002800DB101A002900DB511A81427047B3
:1057E00010B5202A04DB0146203A9140002010BD6C
:1057F000914020239C1A0346E3401943904010BD7A
:1058000010B5202A04DB0846203AD040002110BD04
:105810000B46D340D0402024A21A91400843194699
:1058200010BD10B5202A06DBCB170846203A1041E0
:10583000C1170B4306E00B461341D0402024A21AA7
:1058400091400843194610BD002904DA401C490064
:1058500001D140084000704770B40024050C05D108
:105860001024000402D1002921D01124050E01D1F9
:1058700000020834050F01D10001241D850F01D15C
:105880008000A41C002801DB4000641C002908D013
:1058900020252E1B0D46F540A14000D001212943B3
:1058A000084301061B1B000ADB1D02D5002070BC4B
:1058B0007047DB05181880180029F8DA401C4900E9
:1058C000F5D170BC40084000704710B5002B08DAD5
:1058D0000024401C614192185B411A4301D14008E9
:1058E000400010BDF0B51FB482B005460C0003D0D7
:1058F000084604F049FD02E004F046FD203002466F
:10590000009021462846FFF76BFF049B059A04464A
:105910000F4618431143084314D0184610431BD0B8
:10592000009840210A1A18460599FFF769FF0546B5
:105930000E46009A05990498FFF752FF084305D0D8
:10594000012004E02046394607B0F0BD0020C11711
:1059500005430E432C43374300990E986305401AC4
:105960007905E40A00220C43FD0A0A3002D5002022
:105970000146E9E70105101969410C9C0D9D0019CC
:105980006941FFF7A2FFDFE74A0009030123090B82
:105990001B0519430A4B10B5520D9A4202DA00203A
:1059A000014610BD064B34339A4203DC9A1AFFF7C6
:1059B00027FF10BD034BD218FFF712FF10BD0000E8
:1059C000FF030000CDFBFFFF064C0125064E05E05E
:1059D000E36807CC2B430C3C98471034B442F7D310
:1059E000FFF772FBA8BB0008C8BB000870B58C1895
:1059F0000578401C6B075B0F01D10378401C2A110E
:105A000006D10278401C03E006780E70401C491C49
:105A10005B1EF9D12B0705D40023521E0DD40B7049
:105A2000491CFAE70378401CCB1A921C03E01D784E
:105A30000D70491C5B1C521EF9D5A142D8D3002021
:105A400070BD000038B50446064805490068FFF7F8
:105A50004FFB604300E0401E00900028FBD138BDA2
:105A600040420F0030010020F8B50446006881680C
:105A70008907890F012902D10168C90722D18168EC
:105A8000114A10261140012500290ED181682943B1
:105A900081600120FFF7D6FF00F0A4FF07460CE06D
:105AA00000F0A0FFC01B0A2807D9606D3043606575
:105AB000A06D2843A0650120F8BD20680068C043A0
:105AC000C007EDD10020F8BD1700008010B50023FD
:105AD0001A4603E0845CE3189BB2521C8A42F9D355
:105AE000D84380B210BD000010B5034800F036FD69
:105AF000024800F033FD10BD30160020E8150020EC
:105B000030B5446C1C252C400125A540046C656013
:105B1000046863608368102B036803D09960006891
:105B2000C26030BD9A600068C16030BD1449012078
:105B300048720A4602205E32507203203C3A50728C
:105B400004200E3A50720F480D4B00780870223135
:105B50000870203108770C495A1C08785871497828
:105B6000997123331871597120331877597710754B
:105B700051751A461E321075517510765176704760
:105B800064110020DF0000200001002010B503F0A8
:105B90004BFD202003F0F4FD012005F09BFB0020CD
:105BA00003F0EEFD044805F039FA044805F0E8FC7E
:105BB000002005F01DFD10BDC800002083800000FE
:105BC000F8B505200121000700F0F8FE0025174C6C
:105BD000002800D06560164E0221304600F0EEFE2F
:105BE00000281BD1012020701248808F00280ED081
:105BF0000127BF0200223946304600F0ECFE0A20A1
:105C000005F0BEF901223946304600F0E4FE0A48AC
:105C1000656000880A21484308490880012000F097
:105C200005FE022000F002FEF8BD00001C0100206D
:105C300000040050640D0020EC000020FE00002055
:105C40007047000010B5084900224A6107494B68B7
:105C50004C1523434B604B68082423434B60C00919
:105C6000C001026010BD0000781600200020024034
:105C70007FB500250C460646039500F0A7FDE00918
:105C8000029003A901960095684600F037FD0028B0
:105C900004D000F06FFD002004B070BD00F06AFD7C
:105CA0000120F9E710B5002302E0C45CCC545B1C72
:105CB0009342FAD310BD000010B5214A002190692B
:105CC000C305204804D54169022319434161911558
:105CD00093699B0505D5436901242343436163020E
:105CE000194393695B0505D5436908242343436140
:105CF000E301194393691B0505D543690424234334
:105D000043616302194393699B0405D543691024D9
:105D1000234343616302194393699B0304D5446998
:105D200020231C43446119439369DB0305D5436970
:105D3000402423434361A0020143916110BD000050
:105D4000002002407816002070B5054600F04AFE9B
:105D50000646184C0AE0681C08D0002D04D000F05C
:105D600041FE801BA84201D9032070BDA069C00775
:105D7000F1D1A069800701D50220A061A069C0050A
:105D800011D4A06980050ED4A06940050BD4A06988
:105D9000000508D4A069800405D4A069800302D45A
:105DA000A069C00303D5FFF787FF012070BD002065
:105DB00070BD000000200240F8B5174600260546D9
:105DC0000C4600F003FD09E029460220226800F09D
:105DD000DFFC002804D1241D2D1D361DBE42F3D347
:105DE00000F0C8FCBE4201D20020F8BD0120F8BD81
:105DF00010B5084902460020054B497905E04400EA
:105E00001C5B944203D0401CC0B28842F7D310BD43
:105E10008C1200205800002010B500F0D4FD10BDF9
:105E200010B5094800F0FEFF80B2FFF727FC074AD3
:105E3000074BFFF71DFB0022064BFFF781FBFFF727
:105E400063FC80B210BD00009C140020F853E3A551
:105E50009B843E4000408F4070B5354C3348217FD5
:105E60000175617F417533490A7802764978417638
:105E70002E490520133148720A2005F071FB7D2060
:105E8000C00005F087FB2949002213310C2005F0E2
:105E900051FC00210C2005F05FFC022005F0B0FB56
:105EA000254D00210F2005F0DBFA2842E062F8D0F2
:105EB000E06A411C38D0400435D58122D20100214E
:105EC0000F2005F00CFC0021102005F0C9FA410656
:105ED0001648490E0022633005F0F8FA134D633579
:105EE000687A05281FD102221249681DFFF76AF956
:105EF000002818D10E48AE7C66710422691C44301B
:105F0000FFF73CF929461331084672000D4651301F
:105F1000FFF734F96079294642000448DF30FFF783
:105F20002DF90320207070BD04F08CFAC5110020FB
:105F3000580000200001002000D0272410B5084898
:105F400000F096FA0A21064800F032FA044800F000
:105F50001DF9800503D5024800F01AF980B210BD82
:105F600040140020F8B52F4D00220121284600F0F2
:105F700032FDFFF7E3FFFFF766FB2B4E3146FFF7DD
:105F800087F92A4C0122A0601146284600F023FD23
:105F90002749A068002588423EDB2078254F00284D
:105FA00015D02570FFF7CAFFFFF74DFB3146FFF70D
:105FB0006FF9A060FFF7C6FB00223B46FFF74AFAE5
:105FC00000221D4BFFF754FAFFF7E4FB6060A06866
:105FD000FFF7B8FB00223B46FFF73CFA174A184B85
:105FE000FFF746FA06460F466068FFF7ABFB134A19
:105FF000144B5242FFF73CFA32463B46FFF786F914
:10600000FFF7C8FB10496060884201DD616004E071
:10601000FF21C905C84200D365606068FFF73CFBFB
:10602000C0B2F8BD0004005000401B443000002006
:106030000000604000000C4000E064403333333324
:1060400033B33040CCCCEC3F0000C842F8B5054635
:1060500004464035287C0026012808D001202874F9
:10606000206881688907890F01290ED101E002208B
:10607000F8BD0168C90708D0606D2021084360653C
:106080000126002028743046F8BD616DFF220132E0
:106090009143022211436165C1688907890F00910C
:1060A000C16889088900C16020688168920711432E
:1060B000816000F097FC07460EE000F093FCC01BE7
:1060C0000A2809D9606D02218843102108436065C0
:1060D000002028740120F8BD206880680028ECDBCF
:1060E0002068C168009A1143C160606D800880001B
:1060F000401C6065C5E70000F8B506460D46403611
:10610000317C01290DD00121317401688A68520760
:1061100009D5416D202211434165002030740120D2
:10612000F8BD0220F8BD174B6A68D80547109A429F
:10613000154C8A6A2B6812D05B035B0B1A438A6288
:106140002968490305D5A1680143A1600A20FFF72A
:1061500079FC2868800312D5A06838430EE05B0301
:106160005B0B9A438A622968490302D5A16881437F
:10617000A1602868800302D5A068B843A060002011
:106180003074F8BD0110000000270140406D7047D9
:106190000068006C7047000070B5040006D0606DA8
:1061A000264600254036002802D006E0012070BDBA
:1061B000A5653574204600F0D3F8606DC00603D4A1
:1061C00021688868400705D5606D10210843606527
:1061D0003574EBE7606DFF220132904302221043D9
:1061E000606588688207920F5B48012A02D10A68BD
:1061F000D2072BD1032362689B079A4205D05B42EA
:106200009A4202D05B009A4209D10A699200920830
:106210000A6121680A6963681A430A610CE00A6925
:10622000920092080A6181680F2292049143816072
:1062300081686268114381602168CA6818239A43A3
:10624000CA602168CA68A3681A43CA6081680122CB
:106250005206914381608168A28E5206114381608B
:1062600020688168C90004D48168012212071143A3
:1062700081602068C168394A1140C1602069E168C5
:10628000022825D000200143204620300278037BDD
:1062900052035B001A431143226B1143A26992031C
:1062A0001143E269D20311432268D3681943D160D4
:1062B000616A0A46FF3AC23A05D0A26A11432268CF
:1062C000D3681943D16042780121012A02D00BE042
:1062D0000420D8E70078002823D0606D20221043E6
:1062E0006065A06D0843A065E06B012820681FD0A1
:1062F0000169C90703D001694908490001612068A3
:106300004169C908C900416120684169A26B114314
:106310004161A565606D80088000401C60650020BB
:1063200070BD2068C26801231B041A43C260DBE70A
:106330000269FF239B009A43026120680269236C73
:10634000A66C1A43636C33431A43026120680269E6
:106350000A430261D3E70000002701401902FEFF53
:1063600010B586B0044614216846FEF720FF0E499A
:106370002068884216D10D48416B42151143416394
:10638000C16A01221143C162C06A6946104005908A
:1063900002200090032001900020029005200007B9
:1063A00000F050FA06B010BD002401400010024079
:1063B000F8B504464069254640350E4608280BD0FE
:1063C0002068C068C00709D0606D2021084360655F
:1063D000002028740120F8BD082700E00C2700F0F9
:1063E00001FB009011E0701C0FD0002E05D000F0D2
:1063F000F9FA0099401AB04207D9606D04210843A8
:106400006065002028740320F8BD206800683842C9
:10641000E9D0606D01214902084360652068C168C8
:1064200009058A0F0C21002A1BD12022125D002AA7
:1064300017D10268120714D5826853070122002B76
:1064400008DB43688B434360606D1302984310433D
:10645000606506E0606D202318436065A06D104301
:10646000A065A069002801D1206801600020F8BD66
:1064700070B50446216800208968490721D4254663
:106480004035297C01291CD001212974E1690129A9
:1064900004D02046FFF7E8FA002811D1616D0A4ABE
:1064A0001140FF220132114361650021A165297469
:1064B00022681C21116021688A6804231A438A60BB
:1064C00070BD022070BD0000FEF1FFFF30B5014637
:1064D00020314A790023022A04D00422C2630B71BE
:1064E000012030BD026814680E25AC4314600268B8
:1064F0001468640864001460446C1C221440012277
:106500001546006CA54045604A7118460B7130BDB8
:1065100070B50024014620314A79022A03D00421B3
:10652000C163012418E0026813680E25AB431360B1
:10653000026813685B085B001360436C1C22134005
:10654000012215469D40036C5D604A7100220A716C
:10655000816B002900D08847204670BDF0B4016CE3
:106560000D6801680C68466C1C2304221E40174607
:10657000B7402F420ED067070CD50C68A40602D492
:106580000C6894430C60416C19408A40016C4A606D
:10659000016B1AE00227B74002462F402032002F3D
:1065A00017D0A70715D50C68A40605D40C680A25D2
:1065B000AC430C6001215171446C02211C40036CFE
:1065C000A140596000211171C16A002918D0F0BCA6
:1065D00008470827B7402F4212D0240710D50C686F
:1065E0000E25AC430C60446C01211C400B46A340BB
:1065F000046C6360C163517100211171416BE4E768
:10660000F0BC704770B504003CD01F4825681421C9
:106610002818FEF76DFD800060641C48206402218C
:10662000204620300246417129681948E36801403C
:10663000A06866691843236933431843A369184364
:10664000E3691843236A1843084328600121A068BE
:106650008903884210D00D488030836A656C1C2104
:106660000D400F26AE40B3438362656C63680D40F6
:10667000816AAB400B4383620020E06301215171CA
:10668000107170BD012070BDF8FFFDBF0000024019
:106690000F80FFFFF8B504468C46203001790025B5
:1066A000012909D00126067141790027012905D069
:1066B000077102252846F8BD0220F8BD022141716C
:1066C000E763206801684908490001606146204687
:1066D000FFF716FA206B00282068016801D00E220F
:1066E00005E0042291430160206801680A221143F9
:1066F00001602068016831430160DBE7F8B51A4E9C
:106700000546307C0F46012807D001203074174819
:10671000FFF71AFB010002D021E00220F8BD0020A3
:10672000C04338606C6814E02046FFF78BFA0F48CE
:10673000FFF70AFB01460E48426808239A4342606D
:10674000426843159A434260002901D03C6006E04C
:106750008034A8686A68C0018018A042E4D800208C
:1067600030740846F8BD00007816002050C30000C1
:1067700000200240054841680222114341604168FF
:1067800001221143416000207047000000200240B8
:10679000F8B50C4C1646207C0F46012808D0012085
:1067A00020740948FFF7D0FA0025002802D006E03F
:1067B0000220F8BD65613E600348FFF7C5FA257405
:1067C000F8BD00007816002050C300001148416851
:1067D000C9070BD0EFF3108172B60F4AC2600F4A9F
:1067E000C26081F310884168C9070ED141688907EA
:1067F0000DD5EFF3108172B6094A0261094A0261B0
:1068000081F310884068800701D50120704700207F
:106810007047000000200240EFCDAB890504030261
:10682000BFAE9D8C161514137047000010B50449B7
:106830004A69024202D04861FFF7F6FF10BD00002E
:1068400000040140FCB500230124A2E027462A46AB
:106850009F403A406FD04D68012D05D0022D03D0E6
:10686000112D01D0122D16D185680326AC465D008E
:10687000AE46AE406546B543AC46CE687546AE40C2
:1068800065462E43866046680D79BE43ED06ED0FE2
:106890009D4035434560C6685F000325BD40AE4658
:1068A000AE4335468E68BE402E43C6604E68022E0B
:1068B00001D0122E14D1DE08B60036180196366AC1
:1068C0005D07B446EE0E0F25B54000966646AE4312
:1068D000B4460D69009EB54066462E43019D2E626A
:1068E00006687546AE430D79AD07AD0FBD40354323
:1068F00005604D68ED004BD5294D6E6B26436E63E8
:106900009E08284DB6007519AC46AD689E07360F37
:106910000F27B740BD4305273F07B84201D10027E5
:1069200015E0214FB84201D1012710E01F4FB842B6
:1069300002D102270BE02BE01D4FB84201D1032703
:1069400005E01C4FB84201D1052700E00627B740FB
:106950002F436546AF60184D2E684F689643FF037E
:1069600000D516432E606E684F689643BF0300D56E
:1069700016436E60AE684F689643FF0200D516431B
:10698000AE60EE684F689643BF0200D51643EE60D6
:106990005B1C0A681546DA4000D057E7FCBD0000D2
:1069A00000100240000001400004005000080050A8
:1069B000000C0050001C0050000401400069084019
:1069C00000D001207047426913460B401B049143DD
:1069D0000B4383617047002A01D081617047816257
:1069E00070470000014880687047000024010020C3
:1069F000024881680278891881607047240100206C
:106A000010B5084800240168402211430160204667
:106A100000F00AF8002801D0012401E000F04CFA4F
:106A2000204610BD0020024070B504460D4D7D206B
:106A30002978C000FEF75CFB01460B480068FEF7B2
:106A400057FB00F035FF002809D1042C07D20022A3
:106A50002146401E00F058FA00206C6070BD0120F5
:106A600070BD0000240100203001002070477047F5
:106A7000F8B5644CA078401CA07001202071A08B58
:106A8000401CA0836048008802F036FE5F48C08842
:106A9000FEF7D9FD5E49FEF7FBFB5E4D0646296811
:106AA000FEF79DFB28600120A16AC005814201DA42
:106AB000084603E03046FEF7E7FBA062FF21C90568
:106AC0000025C84200D3A562607800280BD10221BE
:106AD0005148FFF773FF02005049514817D0002278
:106AE000FFF779FFA56302214B48FFF767FF0028F6
:106AF00055D0A563454FB88AFEF7A5FD454E3168D0
:106B0000FEF764FE5DD24749012008705BE0012278
:106B1000D1034348FFF75FFF3C48C088FEF793FD71
:106B20003B49FEF7B5FBA16BFEF759FB3E49A0635D
:106B30008842D8DD35480127F926403000900A21E7
:106B40003046FEF7D5FA002903D134493448FFF71F
:106B500063F902213048FFF731FF002801D00027F8
:106B600001E0002F12D102212B48FFF727FF002858
:106B70000CD104F02BFF00990120888004F084FFE1
:106B8000642004F0FDF92A492848C8600A2004F06E
:106B9000F7F93046761EF6B20028D0D1A3E71B489D
:106BA000C088FEF750FD1A49FEF772FBA16BFEF795
:106BB00016FB2049A06388429CDB1D491B48C86026
:106BC00098E718480570788F401EFEF731FD316850
:106BD000FEF7FCFD06D86079002803D01649012095
:106BE000087001E014480570788FFEF72CFD3168BD
:106BF000FEF7ECFD04D26079002801D004F0AAFE73
:106C0000F8BD0000DC00002072000020640D0020B0
:106C100000007A44200100200004005000800000A1
:106C2000000000505E000020000040400400FA0513
:106C300000ED00E00000A0406B000020704770B540
:106C4000040010D0022025462035A873204601F00C
:106C5000E5FCA87B032805D0204600F0B9F8002009
:106C6000A873687370BD012070BD7047704710B580
:106C7000044600680168C943C90708D18168C9434F
:106C8000C90704D1012141602046FFF7F1FE2068C9
:106C90000168C943890708D48168C943890704D4B6
:106CA000022141602046FFF7E1FE20680168C943E8
:106CB000490708D48168C943490704D404214160C5
:106CC000204600F0F7F820680168C943090708D496
:106CD0008168C943090704D4082141602046FFF7B1
:106CE000ADFF20680168C943C90608D48168C9435B
:106CF000C90604D4102141602046FFF7B8FE206881
:106D00000168C943890608D48168C943890604D447
:106D1000202141602046FFF7A9FF20680168C94390
:106D2000490608D48168C943490604D4402141601A
:106D30002046FFF79AFF10BDF8B5040005D02546A0
:106D40002035A87B002802D006E00120F8BD0020F5
:106D50006873204600F04EF80220A8732068C268CD
:106D600084466368012B01D106208243164861697D
:106D7000814202D0072040038243002B01D1D8205A
:106D800082431248A668024018463043676A266A62
:106D90003E433043A66A30431043002B02D0012B00
:106DA00004D005E02369E2691A4300E0E268104379
:106DB000054A914202D0A269114308436146C86066
:106DC0000120A8730020F8BDFFFF0000F8F119FFB3
:106DD00010B500680549884207D10548816B490014
:106DE000490881630D2000F073F810BD007C00405D
:106DF0000010024010B50068084988420CD10848CC
:106E0000816BC20411438163002201210D2000F037
:106E10007BF80D2000F06CF810BD0000007C0040F5
:106E2000001002400068C06970470000F8B50446D1
:106E30000220254620351746A8731D480268C30462
:106E40001A4302602068C2689B121A43C26020681D
:106E500002690126324302612268102050602068D6
:106E600081611021204601F049FC03281FD02168D0
:106E700008204860206847610821204601F03EFC58
:106E8000032814D0204601F0C9FBA87B03280ED0AC
:106E90002068816831438160206801693143016164
:106EA00020680169042211430161AE730020F8BD1E
:106EB00000040140704700000448416B0122114367
:106EC0004163816B020411438163704700100240EB
:106ED000002809DBC106C90E01208840034908606B
:106EE000BFF34F8FBFF36F8F7047000080E100E06A
:106EF000002805DBC106C90E012088400149086051
:106F00007047000000E100E010B503F079FA10BD11
:106F100002494A6882434A6070470000007000409E
:106F200002480168821511430160704700700040FB
:106F300002494A6802434A607047000000700040FE
:106F400005480168022211430160044801690422D6
:106F50001143016130BF70470070004000ED00E058
:106F6000F0B5154A1368154D54152D6A2340ED07E9
:106F7000ED0F002B04D0002D02D01668A64316603A
:106F80001668B608B600064316600D480769042661
:106F90003743076101290DD040BF20BF20BF0169E1
:106FA000B1430161002B04D0002D02D010682043B2
:106FB0001060F0BD30BFF2E70070004000000140FB
:106FC00000ED00E0F8B5044600780027534D800638
:106FD00071D5524E403EB06BC00004D4B06BA905D1
:106FE0000843B06301274E480168C90511D4016800
:106FF000821511430160FFF7F5FC009005E0FFF7F3
:10700000F1FC0099401A642837D845480068C0054B
:10701000F5D532680321090560680A4001409142B4
:1070200008D08103890F032904D13168890301D570
:107030000120F8BD2A69032109040A4022D0084032
:1070400090421FD0207880061CD528692A69884381
:107050000121C9040A432A612A698A432A612861F5
:10706000C0050FD5FFF7BEFC009008E0FFF7BAFCA3
:107070000099411A2B48814201D90320F8BD2869A3
:107080008005F3D561688803800F032805D1326835
:107090000005824301400A43326028690322616887
:1070A0001204114008432861002F04D0B16B012065
:1070B00000078143B1632078C00705D0E868A16864
:1070C000800880000843E8602078800705D5E868DC
:1070D0000C218843E1680843E8602078400706D522
:1070E000E86803218902884321690843E860207821
:1070F000000706D5E868032109038843616908434E
:10710000E8602078000606D5E868032189048843F2
:10711000A1690843E8600020F8BD0000401002406B
:107120000070004088130000F8B50E46050038D006
:107130005E480068C007C00FB04214D25B4C2068A4
:107140004008400030432060FFF74CFC074605E054
:10715000FFF748FCC11B564881427AD82068C00717
:10716000C00FB042F4D12878524C800705D5E068B2
:10717000F0218843A9680843E0602878C00752D00E
:107180006868022806D0032807D0216801280AD0A1
:10719000890504E02168890301E02168890100294B
:1071A00003DB0120F8BD4907F9E7E1688908890098
:1071B0000143E160FFF716FC0746686802280AD021
:1071C000032814D001281ED029E0FFF70BFCC11BB7
:1071D000374881423DD8E0680007800F0228F4D18B
:1071E00021E0FFF7FFFBC11B3148814231D8E06845
:1071F0000007800F0328F4D115E0FFF7F3FBC11B54
:107200002B48814225D8E0680007800F0128F4D17F
:1072100009E0FFF7E7FBC11B2548814219D8E06868
:107220000007800FF5D121480168C907C90FB14295
:1072300017D901684908490031430160FFF7D2FBC3
:10724000074608E005E0FFF7CDFBC11B1848814267
:1072500001D90320F8BD15480068C007C00FB0422F
:10726000F1D12878400706D5E06807210902884354
:10727000E9680843E0602878000707D5E06807213F
:10728000C90288432969C9000843E06000F03AF860
:10729000E168094A0906090F515CC84007490860BE
:1072A00007480068FFF7C0FBF8BD0000002002405F
:1072B000881300000010024086BB00083001002047
:1072C00028010020044805490068C968044A4905A6
:1072D000490F515CC8407047300100200010024047
:1072E0009FBB0008044805490068C968044A89042E
:1072F000490F515CC8407047300100200010024027
:107300009FBB000870B51A4AD3681A490C20184070
:107310008D0004280CD04E00082810D00C2810D066
:1073200050680004410F0120C003491C884070BD13
:107330001068C00601D5084670BD284670BD3046AD
:1073400070BD98020C4C000F205C1B029C0FD36890
:10735000641CDB0301D5314603E01268D20600D479
:10736000294603F028F822460023FDF7D7FE70BD1A
:107370000010024000093D0096BB0008FEB5050064
:107380007ED0FE4CE7680C20E66807400120000430
:1073900006402878C00747D0082F05D00C2F0AD107
:1073A00001200004864206D1206880033CD568682D
:1073B0000028E5D038E0012069680004814203D14B
:1073C00021680143216011E0052301221B0492047E
:1073D0009942216802D111432160F1E78143216084
:1073E000216801400091206890432060686800286F
:1073F0000DD0FFF7F7FA009005E0FFF7F3FA0099D8
:10740000401A64287BD820688003F6D50CE0FFF78B
:10741000E9FA009005E0FFF7E5FA0099401A6428C0
:10742000F0D820688003F6D42878800756D5092341
:10743000E868042F0DD00C2F01D1002E09D00028B0
:107440003CD02168994301432160FFF7CBFA0646FF
:1074500028E02168490701D5002891D061681F22E2
:10746000120291432A691202114361602168994313
:1074700001432160FFF746FFE16809060A0F00E0BB
:107480008BE1BF49895CC840BE490860BE480068BE
:10749000FFF7CAFA002873D120E0FFF7A3FA801B98
:1074A0000228AFD820684007F7D560681F2109027D
:1074B000884329690902084360600FE0206840089A
:1074C00040002060FFF78EFA064604E0FFF78AFAD4
:1074D000801B022896D820684007F7D42878C00679
:1074E00060D5002F0CD0A86900284AD02068FF2161
:1074F000013108432060FFF775FA06462EE0C1E02F
:107500002068800502D5A8690028A6D060680721F8
:1075100049038843296A084360606068297F000244
:10752000000A090608436060286A410B0120C00375
:10753000491C8840E16809060A0F9149895CC840E6
:107540009049086090480068FFF76EFA002817D14C
:1075500028E0FFF747FA801B0228A2D820688005A0
:10756000F7D56068072149038843296A08436060AA
:107570006068297F0002000A09060843606011E084
:10758000E2E02168FF20013081432160FFF72AFA01
:10759000064604E0FFF726FA801B022872D820680E
:1075A0008005F7D42878794E000724D5686900282B
:1075B000306910D0012108433061FFF713FA0090C1
:1075C00005E0FFF70FFA0099401A02285AD83069EF
:1075D0008007F6D50FE0400840003061FFF702FA5F
:1075E000009005E0FFF7FEF90099401A022849D8FB
:1075F00030698007F6D42878400766D500200290CD
:10760000A06BC00006D4A06B012109070843A0634A
:10761000012002905E480168C90511D401688215F5
:1076200011430160FFF7DEF9009005E0FFF7DAF99A
:107630000099401A642825D855480068C005F5D53A
:10764000FF20AA680130824203D1316901433161D0
:1076500011E001218902002A07D005231B029A426A
:1076600003D132690A433261EFE732698243326102
:10767000306988433061A868002810D0FFF7B2F95C
:10768000009008E05FE0FFF7ADF901460098091AA5
:107690004048814257D830698005F4D50DE0FFF7A6
:1076A000A1F9009006E0FFF79DF90099411A3948C9
:1076B000814248D830698005F5D40298002804D06A
:1076C000A06B012109078843A063686A002866D07F
:1076D0000C2F3ED0012636060228206805D0B04384
:1076E0002060FFF77FF905462FE0B0432060FFF7E9
:1076F00079F9074604E0FFF775F9C01B022822D884
:1077000020688001F7D4E96AA86AE2680843296B17
:10771000FD231B049A4311430843E0602068304373
:107720002060FFF75FF9054604E0FFF75BF9401BB7
:10773000022808D820688001F7D530E0FFF752F919
:10774000401B022801D90320FEBD20688001F5D42A
:1077500025E00128F8D0E06801210904AA6A014067
:1077600091421AD10F218904EA6A0140914214D151
:10777000032189050840296B88420DE00010024072
:1077800086BB000830010020280100204010024084
:10779000007000408813000001D00120FEBD0020D1
:1077A000FEBDF8B504000ED0FF27606A053700253E
:1077B00000280AD02561656126464036A562707CA6
:1077C000002807D00AE00120F8BD6068B842F3D075
:1077D000E561F1E73574204600F03EF8022171744E
:1077E0002068026840239A4302602123A2686068EF
:1077F0009B021A4038401043E3688A021340184342
:1078000023690B40217D1843C907C90F0843A169AB
:10781000931019400843E169382319400843216A4D
:10782000802319400843A16A930019400843216846
:107830000860A0690421000C0840616A1023194007
:107840000843216848602068C1699143C16165654A
:10785000012070740020F8BD10B586B004461421D4
:107860006846FDF7A4FC10492068884219D10F48EA
:10787000416B821411434163C16A01221143C16209
:10788000C06A002110400590E02000900220019085
:107890000320039002910491052069460007FEF73A
:1078A000D1FF06B010BD00000030014000100240C2
:1078B000094910B5401E884201D9012010BD074C6E
:1078C00060610321081F02F09BFD0020A0610720DA
:1078D0002061002010BD0000FFFFFF0000E000E07D
:1078E000F0B502462032137E012B1ED001251576FD
:1078F0000223537606687468B3687027BC430F6828
:10790000274377600068AC07A04205D0084CA0422E
:1079100002D0084CA04204D180244968A3431943F3
:107920008160557600201076F0BD0220F0BD000089
:10793000000801400014014070B5050005D02C4638
:107940002034607E002802D006E0012070BD0020B7
:107950002076284600F010F802206076291D28685D
:1079600001F092FF0120A077A076E0762077607783
:107970006076002070BD0000006801218907884200
:1079800004D10348816B01221143816370470000D9
:1079900000100240F8B5054604462035287E01282F
:1079A00017D001262E760220687622689068772705
:1079B000FF23B8431B02984390600A68502A31D0D5
:1079C0000EDC202A4BD006DC002A48D0102A3AD1FF
:1079D00045E00220F8BD302A41D0402A33D136E0BC
:1079E000602A27D0702A12D001200003121A2AD050
:1079F000824228D1CB684A688968206801F07DFFFF
:107A00002068816801229203114381601BE0CB68EA
:107A10004A688968206801F070FF216888683843E7
:107A2000886010E0CA684968206801F0E0FF5021D2
:107A3000206806E0CA684968206801F0E9FF602113
:107A4000206801F065FF6E7600202876F8BDCA68D0
:107A50004968206801F0CBFF40212068F1E711461A
:107A60002068EEE710B586B0044614216846FDF79D
:107A70009EFB012120688907884212D10A49CA6AFF
:107A800002200243CA62C96A019001400591410285
:107A90000091002102910391049069460348FEF78A
:107AA000D1FE06B010BD00000010024000040050DE
:107AB000F8B5064604462036307E0D4601280BD028
:107AC000012008273076002A08D0042A16D0082A78
:107AD0002AD00C2A4DD137E00220F8BD206801F0F1
:107AE0001FFF206881693943816120688169042210
:107AF0009143816120688169EA6812E0206801F0A1
:107B000027FF206881690122D20211438161206828
:107B10008269012189028A43826120688169EA6859
:107B200012021143816124E0206801F02AFF2068DD
:107B3000C1693943C1612068C16904229143C161AF
:107B40002068C169EA6812E0206801F035FF20680A
:107B5000C1690122D2021143C1612068C2690121B9
:107B600089028A43C2612068C169EA68120211432E
:107B7000C16100203076F8BD70B5050005D02C46F7
:107B80002034607E002802D006E0012070BD002075
:107B90002076284600F00FF802206076291D28681C
:107BA00001F072FE0120A077A076E0762077607762
:107BB0006076002070BD704770B505462C460220E7
:107BC0002034002908D004290BD008290ED0627F68
:107BD000012A10D0012070BDA27E012AFAD1A07620
:107BE0000AE0E27E012AF5D1E07605E0227F012A53
:107BF000F0D1207700E060770122286801F070FE64
:107C00000122286892070121904205D0074A90423C
:107C100002D0074A904204D182685207520F062AC6
:107C200002D002680A430260002070BD00080140D3
:107C30000014014070B504460D460068002201F0B2
:107C40004FFE2068016A0C4A114203D101684908BD
:107C50004900016001202034002D06D0042D06D0FB
:107C6000082D06D06077002070BDA076FBE7E07697
:107C7000F9E72077F7E7000011110000704770471F
:107C800070470000F8B502680446D069116896682C
:107C9000814B05461D402023002D6CD0F7077F4DFA
:107CA000FF0FBC460D402F4379D02546C7078035CE
:107CB000002F06D0CF0504D5012717622A683A4362
:107CC0002A60820708D5F20706D0276802223A62A6
:107CD0002A6804273A432A60420708D5F20706D0EB
:107CE0002668042232622A68022632432A6002078A
:107CF0000AD50A461A406646324305D0266808224D
:107D000032622E6816432E60020508D54A0106D558
:107D100001222668D20232622A681A432A602A683F
:107D2000002A30D0800606D5880604D5616E002969
:107D300001D020468847286821688968490602D40E
:107D40002821084225D0204602F067F82068816883
:107D5000490619D5826840218A438260206F002835
:107D600012D04F498163206FFEF7D2FB00280AD062
:107D7000206F816B06E0850611D58D060FD5616EEB
:107D800077E020468847F8BD2046FFF779FFF8BD29
:107D900005E02046FFF774FF00202860F7E7256E16
:107DA000012D56D1C50654D5CD0652D510261662E2
:107DB0002068816825464906403500292ADA226F65
:107DC000116849680904090CE1D02F8B8F42DED974
:107DD000698311680968890617D4016832019143E3
:107DE00001602068816849084900816020688168D5
:107DF000402291438160E36700202066206801688B
:107E0000B1430160206FFEF761FB288B698B401A3C
:107E100081B21AE0298B6A8B891A6A8B89B2002A8F
:107E2000B5D00029B3D00268FF252135AA430260EE
:107E300020688268520852008260E3670020206652
:107E4000606620680268B24302602046FFF716FFB2
:107E50009DE7C50208D5750206D501200005106210
:107E60002046FFF70CFF92E7050605D50D0603D562
:107E7000A16E002985D18AE7400688D5480686D5B7
:107E8000116820464024A143116083670021816668
:107E900000F043F97BE700000F0800002001000418
:107EA000419D000810B5040003D0A06F002802D047
:107EB00007E0012010BD002174200155204600F08C
:107EC00027F82420A067206801684908490001605C
:107ED000204601F0F5FF0128ECD0606A002802D0AE
:107EE000204601F00DFE206841680922D20291432C
:107EF0004160206881682A2291438160206801687E
:107F0000012211430160204601F060FE10BD000017
:107F1000F0B587B0064614216846FDF748F92C49AC
:107F20003068884251D12B48416B012292031143A2
:107F30004163C16A01221143C162C06A0025104039
:107F400005900320400200900220032701A9A1C14F
:107F500004200490052069460007FEF773FC1F4CBF
:107F60001D48A560E56081C48027E560A7602020EA
:107F7000256160610002A0611848083CFEF742FBE1
:107F8000002801D0FDF75CFE3467A662144C12484D
:107F90002146143820600320606010200831A1C100
:107FA0006561A561E56120462562FEF72BFB00288F
:107FB00001D0FDF745FEF466002201211B20A662D8
:107FC000FEF7A2FF1B20FEF793FF07B0F0BD0000F5
:107FD000003801400010024030000240E815002047
:107FE0003016002070B5C36F202B27D100290BD08D
:107FF000002A09D0012483682403A34206D103691F
:10800000002B03D1CB0701D0012070BD03466033A4
:108010001C7D012C12D001241C7500230366084C22
:108020000368A34207D05C68240204D51C680125BC
:10803000AD062C431C6002F043F870BD022070BDF9
:108040000048004070477047FFB50446806F83B01A
:1080500017460D4620285ED1002D0AD0002F08D0EB
:10806000A168C001814207D12069002804D1E80736
:1080700002D0012007B0F0BD204660300090007DA6
:10808000012848D000980121017500208021085165
:108090002120A067FEF7A6FC2646403601903782D5
:1080A00077820120A1680003814202D12069002863
:1080B00005D02F46002500990020087511E0002703
:1080C000F9E700228021204602F040F8002815D16F
:1080D000002F15D02168387888627F1C708A401E76
:1080E0007082708A019B002806980090E9D10022D6
:1080F0004021204602F02AF8002808D00320B9E7E2
:1081000028882168C005C00D8862AD1CE6E72020E4
:10811000A0670020AEE70220ACE7704701490248A3
:10812000C160FDE70400FA0500ED00E070B586B01F
:1081300014216846FDF73BF80F480124418B0029C4
:1081400000D14483408B012805D0022801D100F0E2
:10815000FFFB06B070BD0122084E9502294630464D
:10816000FEF739FC002102910391009501946946C4
:108170003046FEF767FBECE7DC000020000400500F
:1081800010B505242407002204212046FEF723FC15
:10819000002208212046FEF71EFC0A2002F0F7FE0E
:1081A000012204212046FEF716FC0A2002F0EFFE11
:1081B000002204212046FEF70EFC10BD10B5052458
:1081C0002407002204212046FEF705FC0122082195
:1081D0002046FEF700FC0A2002F0D9FE012204210D
:1081E0002046FEF7F8FB0A2002F0D1FE002204210F
:1081F0002046FEF7F0FB10BDF8B500240526074623
:1082000025463607002204213046FEF7E4FB0A200B
:1082100002F0BDFE012204213046FEF7DCFB6006C1
:10822000040E08213046FEF7C9FB002801D0641C6B
:10823000E4B2052002F0ABFE6D1CEDB2082DE1D3D7
:10824000002F03D0FFF79CFF2046F8BDFFF7B6FFD5
:10825000FAE770B5052605463607002204213046A8
:10826000FEF7B9FB0024E80901D0012200E000225A
:1082700008213046FEF7AFFB6806050E0A2002F023
:1082800086FE012204213046FEF7A5FB0A2002F0FB
:108290007EFE002204213046FEF79DFB0A2002F0FC
:1082A00076FE641CE4B2082CDDD370BD10B5052445
:1082B0002407012208212046FEF78DFB012204211C
:1082C0002046FEF788FB002208212046FEF783FBAC
:1082D0000A2002F05CFE002204212046FEF77BFB10
:1082E00010BD10B505242407002204212046FEF706
:1082F00072FB002208212046FEF76DFB0A2002F0E7
:1083000046FE012204212046FEF765FB01220821DA
:108310002046FEF760FB0A2002F039FE10BD70B562
:1083200005252D070024012208212846FEF753FBCE
:10833000062002F02CFE012204212846FEF74BFB0A
:10834000062002F024FE07E0641CE4B2FA2C03D9F4
:10835000FFF7C7FF012070BD08212846FEF72EFB5E
:108360000028F1D1002204212846FEF734FB00202A
:1083700070BD0000F8B501F05BFC01F095FC5848B9
:108380000068C069FDF74CFD564C5749A082898FA3
:10839000564E0025002931D0A26A730354499A42EF
:1083A00002DB02220A7000E00D700A7801218902C6
:1083B000002A05D0012A0ED0022A10D0032A1DD18E
:1083C000608B01282BD0022818D14548082140385D
:1083D000FFF730FC12E0FF22F5329042F0D2608BC2
:1083E00001281AD0022804D008E03046FEF7F3FA3C
:1083F00004E03B4808214038FFF7DEFB0121C902B9
:108400003046FEF7DBFA0127FF0300282AD039485F
:108410000560E079002804D007E00022E5E70122AA
:10842000E3E70120E07101F001FF2078632806D91D
:10843000002208213046FEF7CEFA012205E0012293
:1084400008213046FEF7C7FA00220520394600070A
:10845000FEF7C1FA244C284E4034A08C274F012847
:1084600003D01CE0E5710022EAE725486946088050
:1084700072B680212348FDF7FBFB002804D00222BE
:1084800069462048FDF798FC62B61FA001F06CFF1A
:10849000A58403F0F9FA642002F072FDFE60608C9E
:1084A000012808D110486584058003F0EDFA6420A6
:1084B00002F066FDFE60208C012806D1258403F0C1
:1084C000E3FA642002F05CFDFE600748124A01886E
:1084D000914202D1C088002800D1FE60F8BD0000A2
:1084E00064150020DC000020640D00200004005012
:1084F00069000020200100200400FA0500ED00E0E2
:10850000AAAA0000384A0008BDF8C8EBC9FDBCB6ED
:10851000C4A3CABD0D0A0000AA55000008B5372142
:10852000202000F06EF80321212000F06AF840219D
:10853000222000F066F80821232000F062F8AA212A
:10854000302000F05EF80A48008FC1B2322000F0FF
:1085500058F80221332000F054F85F21202000F069
:1085600050F8684600F006F80A2002F010FD08BD39
:10857000640D002010B501460F2000F021F80028FE
:1085800000D0012010BD10B50446FFF78FFE322049
:10859000FFF75FFEFFF7C3FEE0B2FFF75AFEFFF7FB
:1085A000BEFEFFF783FE3320FFF753FEFFF7B7FE53
:1085B0000020FFF721FE0446FFF793FE204610BD82
:1085C00010B50C46FFF7DFFF2070012010BD70B51D
:1085D0000D460446FFF76AFE3220FFF73AFEFFF72A
:1085E0009EFEE0B2FFF735FEFFF799FE2846FFF743
:1085F00030FEFFF794FEFFF774FE0A2002F0C7FC7E
:1086000070BD10B5FFF7E3FF012010BD10B50248A3
:10861000FEF72DFB10BD00009C140020FEB50446A3
:10862000002772B6334A01688B1804D13248C768F4
:1086300003208004074088680190C868009048695A
:108640008E69002B08D12C4940398B6ACD042B430D
:108650008B628B6AAB438B62014631433CD0254928
:108660002368CB4205D12449CA6803239B049A435B
:10867000CA6025462035002810D021680A690123E8
:108680001A430A61216848610821204600F036F843
:10869000032800D1A873216808204860002E10D05C
:1086A000206801690122114301612068866110215F
:1086B000204600F023F8032800D1A8732168102079
:1086C00048600C482168C14206D10B48C1680322AA
:1086D000920491433943C160206801694908490007
:1086E000016121680198886021680098C86062B6BD
:1086F000FEBD00000084FFBF4010024070B506467A
:108700000B480D46002409490068FCF7F1FC7D2167
:10871000C90048433168401E00D103240B682A4633
:108720009A4301D00028F6D1204670BD204E0000AB
:10873000300100201CB5002116480091144A019117
:108740000260C163120542608160072282630122D8
:1087500002610246C16020321170FF235170C233A2
:10876000436281621173016381610422416342614A
:10877000C161FDF711FD0848009080130190694622
:108780000448FDF7B9FC00210248FDF75FFC1CBD61
:1087900000240140401400200200000408B50848ED
:1087A000016B012211430163006B01211040009015
:1087B00000220A20FEF7A8FB0A20FEF799FB08BD5D
:1087C00000100240F0B587B014216846FCF7EFFCBA
:1087D0004748C26A04210A43C262C26A0A4005923B
:1087E000C16A80263143C162C16A31400591C16AC4
:1087F00001242143C162C16A21400591C16A022559
:108800002943C162C06A22462840059005201C21E8
:108810000007FEF7E0F8012236493748FEF7DBF89B
:10882000002236493448FEF7D6F89121052000226F
:1088300009020007FEF7CFF8314801900027052014
:108840006946029700940007FDF7FCFF0C2000909A
:10885000112001900320039005200297694600072C
:10886000FDF7F0FF10206A46039591C20520694686
:108870000007FDF7E7FF1120019002976946039773
:1088800000941D48FDF7DEFF1E48019069460095E3
:1088900002941948FDF7D6FFE0020090694601975F
:1088A00002951548FDF7CEFF1748694691C1694604
:1088B00011480397FDF7C6FF91200002694691C158
:1088C0000520694600070397FDF7BCFF69460A4883
:1088D000019700960294FDF7B5FF002201210520C3
:1088E000FEF712FB0520FEF703FB07B0F0BD00000A
:1088F0000010024001020000000400500830000097
:1089000000001110000021100832000010B50F4CBB
:108910000D482060FF20053060600020A060E0600E
:1089200020616061E0610121206249026062A16111
:10893000A0620720E0622046FEF733FF206801684E
:1089400040221143016010BD00300140CC140020D2
:1089500010B58AB0002404940594069407940894F2
:108960000121184809940094019402948907039402
:108970000160092184604160046113494461C16060
:10898000FEF7DAFF01200003049004A90D48FFF769
:1089900001F80C48FFF7F0F8089408A90948099471
:1089A000FEF79EFF60200090084801900294082284
:1089B000694603940348FFF77BF80248FFF752F833
:1089C0000AB010BD241500209304000057020000D7
:1089D00000B585B014216846FCF7E9FB0E480D4947
:1089E0000160E1214902416000218160C1600161B3
:1089F00081610C22C1614261016230214162012129
:108A0000090381634900C163FFF74CFA01F008FCD8
:108A100005B000BD0038014064150020704700001B
:108A2000F0B5FF4889B0008801F0ECFB0A2002F0A5
:108A300097FD7D20C00002F0ADFDFA4C0020A07033
:108A4000F949E164617B0C2901D30B216173002595
:108A5000F648E570F64E00783071F649A07909784D
:108A600040000843E17C89000843F071A06AF0707F
:108A7000401CA06260793146B0744200B4310846AF
:108A8000A138FCF77BFB06207072EB4800220078CF
:108A9000B072A07E307330461338217F0175617F3C
:108AA0004175607931464000153002F043FE60792F
:108AB00000214000153002F04FFE022002F0A0FD20
:108AC000F571E573A57201272773E572DB48FEF7A0
:108AD000A9F920840646E5706079FCF7CFFDD84AF5
:108AE000D84BFCF7C5FC02F0E7F90022BB07FCF706
:108AF0000DFCFCF709FE0006C10C881980B2F903D1
:108B00006084884201D3401A6084CF48A0632079F2
:108B1000401C2071C948FEF785F9E083C4480C3039
:108B20000546423540300390BEE1C448FEF77AF96D
:108B3000E083C64E0BE0C148FEF774F980B2E083D3
:108B4000618C884203D3C24A8918884206D3002127
:108B50000F2002F085FC3042E062ECD0E06A411C5C
:108B600021D040047ED58122D20100210F2002F0C5
:108B7000B6FD7D20C00002F00DFD002002F0BFFC1C
:108B80000021102002F06CFC4106A948490E26463F
:108B900000225030A16402F099FCA5485030417A7F
:108BA0000729C1D101E001F04DFC0222A949401D75
:108BB000FCF708FB0028B7D102F01FFEF165B06595
:108BC00002F008FE71663066F0786A46401CF0706C
:108BD00097484D3001791170407950701088049099
:108BE000B18B88427ED19C4E288A30800398808A3F
:108BF00020839248FEF716F9E08302F043FBFF2240
:108C0000216E5204606E0023891858410206080A3A
:108C10001043009040084000010E0002E166A0668B
:108C20008348E36D0A30A26D02F0BCFD6079804993
:108C3000800040181630636E226E02F0B3FD7C484F
:108C4000E36E1230A26E02F0ADFD79490820487241
:108C5000A07C002816D0764802227E495530FCF7C9
:108C6000B1FA00E013E100280CD17148E773C77135
:108C7000A06C6F491638C2B2663108462274EA30D9
:108C8000FCF77CFA60790022800069491C3002F010
:108C900051FD6079002180001C3002F05DFD0098DC
:108CA00002F057FC012002F0ABFC207202216B485D
:108CB000FDF784FE00287DD000215E4801705949EF
:108CC000A8898886EA89CA86616BA16358495031B0
:108CD000CB7C1907090F032900D061741909A1740D
:108CE000002100E077E0217101234E4DA372288717
:108CF0006A87E372208B5A4AFF30C33080B22083E8
:108D000090420BD952428018208330887D22401C2B
:108D100080B2D2003080904200D3318035887D20EF
:108D2000C00029464143208B3D4F0818E06307905F
:108D30003E784C48A673008830214843FCF783FCFA
:108D400000900A2029464143608B30220690504310
:108D5000081AFCF76DFC0099FCF79AFA7F21C90507
:108D6000FCF73DFAFCF798FC80B2761E3880B042E2
:108D700001D10120E072A5841420205EFCF76AFC7A
:108D800006460F46E08BFCF779FC374A374BFCF779
:108D90006FFB054605910798FCF75CFC2A46059B8E
:108DA000FCF758FB32463B46FCF7B0FAFCF788FC70
:108DB000206400E006E0069800F09EFC207A00287F
:108DC00002D07AE0012178E700210F2002F048FB71
:108DD0000006F9D571E0FDF70BF8254A032111547F
:108DE0001049AA898A86EA89CA86214980006039A1
:108DF000421803990190098B11801D4A716B303A1A
:108E000011500B49736E40181630326E02F0CAFCD6
:108E1000F16C706B884200DAF0641549603929E022
:108E2000F8000020580000203F420F00DC00002026
:108E3000D81100201C010020EC0000209C14002010
:108E4000B81E85EB51B8CE3FA086010000D0272484
:108E5000983A000000010020180100200004005092
:108E6000E7030000FC000020F853E3A59B843E408C
:108E70001C130020019A8958814215DD002913D066
:108E8000002811DD0498B083022030700CE03246D7
:108E900000210F2002F023FC6079E178401C814220
:108EA00002D0002002F02BFBE08B618C884200D2C4
:108EB0003BE62B4A89188842FAD8A07A012801D0CB
:108EC0000220A07202F0DEF9264A00210F2002F0F3
:108ED00006FC2079002807D023490A22098851433B
:108EE000814201D200202070E07B00281DD01F4964
:108EF0000B7848788A78022B17D110280CD0C82814
:108F000013D21B4BC91C1818FCF738F902F0BCFD32
:108F1000642002F035F846E6164D28684000000E41
:108F200003D1C878FCF78FFB2860104D00209C3DD2
:108F30002E4621786379183607E04200AF5AB25ABC
:108F4000974200D00221401CC0B29842F5D3054A96
:108F50002170803200210F2002F0C1FB09B0F0BD6A
:108F6000983A000000D02724EC00002028130020AD
:108F7000640D00200401002070470000F0B58DB0A2
:108F8000B44801900020C0430A9000260A2002F055
:108F9000E7FA7D20C00002F0FDFA0020AE4C054645
:108FA000A070AE4FAE480B90AD480022C23885731A
:108FB0000146142002F0BEFB0021142002F0CCFB7D
:108FC000022002F01DFB00210F2002F049FA384276
:108FD000E062F8D0E06A411C18D040047ED58122BE
:108FE000D20100210F2002F07AFB0021102002F0B4
:108FF00037FA41069A48490E0022801C02F066FAB0
:109000009748801C417A022902D007E101F01AFA40
:10901000934802229349C01DFCF7D4F80028F4D1EC
:1090200002F0EBFBE165A06502F0D4FB616620660F
:10903000002E22D10B988C49008A0880884801268E
:10904000801E808A20838948FDF7ECFEE083208B18
:109050008749FF30C33080B2208388420DD949420E
:109060004018814920830888814A401C80B20B3215
:109070000880904201D3002008800B9968468A89B5
:109080000280C989418076490422C91C0846A23859
:10909000FCF774F8FF22216E5204606E00238918D9
:1090A00058410006090A01430846029102F051FAAC
:1090B000029948084000010E0002E166A066684877
:1090C000E36D9638A26D02F06DFB6548636E9238D1
:1090D000226E02F067FB62488E3800E0A0E0E36E8B
:1090E000A26E02F05FFB5E490022A0393C2002F034
:1090F00021FB00213C2002F02FFB012002F080FA2E
:109100002072A0780121401CA0700520C90300072F
:10911000FCF782FE54487D220088D200014602906E
:109120005043228B0A398018E0630C905148007834
:10913000A073049008B2E084002803DA7D21C900FE
:109140004018E0844C48302100884843FCF77BFA03
:1091500005902620205EFCF76BFA0599FCF798F83D
:109160007F21C905FCF73BF8FCF796FA414980B22C
:1091700008800499491E884201D10120E0720298BA
:10918000A0841420205EFCF765FA05910690E08B20
:10919000FCF774FA394A3A4BFCF76AF907910490E4
:1091A0000C98FCF757FA079B049AFCF753F9059BB8
:1091B000069AFCF7ABF8FCF783FA2064608B00F0AA
:1091C0009BFA00990198814210DA00290ED02449B7
:1091D0000422C91C0AA8FBF7D1FF022020702948ED
:1091E0000A2100784843607200980190207A002894
:1091F00005D100210F2002F033F90006F9D58022B5
:1092000000210F2002F06BFA00206D1CEDB260709F
:10921000032D00D2C8E6002E08D017E00120F4E7A5
:10922000194A00210F2002F05AFAF7E7618B17481C
:10923000002902D00288914201D90188618388B255
:109240001349401E09884843124908800A98A083A0
:109250000DB0F0BD3F420F005800002000D0272481
:109260002612002000010020180100209C1400207C
:10927000E7030000F8000020FC000020F853E3A5FD
:109280009B843E40EC00002000902724E800002052
:10929000E6000020E4000020F8B5324930480860BC
:1092A00002F094FB304800F0E7F9304CE0822E48A1
:1092B000801C00F0E1F920832B48001D00F0DCF950
:1092C000608343212A48C900418001464031097921
:1092D000284F0906090E617006D1C7800121C18798
:1092E0000A21418700218187234AC18E1170C18FD5
:1092F0006171818FA171817AE17085880521656234
:109300006181C6883046FBF7F3FEA08101462846FE
:10931000FBF7EEFE8800081885B2164825816843E1
:10932000FCF7ACF9154A164BFCF70AF9FCF7ECF917
:10933000E081658231463846FBF7DAFE208201463D
:10934000C820FBF7D5FE20840120A083FCF768FD30
:10935000A082E2890B490C48FDF768FDF8BD0000CA
:1093600059A2000850000020004F0008DC00002037
:10937000640D0020E803000000000020F853E3A57E
:109380009B843E40FF7F00009C140020F0B5954D6B
:1093900085B001202880944FC820944C3880E07913
:1093A000401CE071C00706D0608B411E618302281B
:1093B00001D2C8206083608B00F09EF90A2002F081
:1093C000CFF87D20C00002F0E5F802218848FDF7C3
:1093D000F5FA002838D00020864980000978874EA9
:1093E00049000843844909780843B072102070721C
:1093F0008348C1887D20C000FBF77AFE70738148E6
:109400007F490078B07330460B308A780270C97893
:109410004170411C7A482030027ECA70407E08713B
:1094200077482230027E4A71407E887100220C39D2
:10943000152002F07FF90021152002F08DF902209D
:1094400002F0DEF8704E03E00120C5E7FEF792FF60
:1094500000210F2002F004F83042E062F6D0E06A0A
:10946000411C7DD040047CD58122D20100210F20F7
:1094700002F035F90021102001F0F2FF41065F48AB
:10948000490E00225030A16402F020F85B4E5036A5
:10949000707A112865D102225C49701DFBF792FE9B
:1094A00000285ED1F01E027969460A704079487042
:1094B000B17A2980C820FBF71BFE3880307B60839F
:1094C000534DB01E008A2880301F808A2083514867
:1094D000FDF7A8FC80B2E0830390208B4E49FF305B
:1094E000C33080B2208388420CD94942401820837F
:1094F00028884949401C80B20B312880884201D31A
:10950000002028802D887D20C000218B68434018D2
:10951000E06301904148067828460A3800B2A673F5
:10952000E084002803DA7D21C9004018E0843888EF
:1095300030214843FCF787F807462620205EFCF7D9
:1095400077F83946FBF7A4FE7F21C905FBF747FEF4
:10955000FCF7A2F880B23149761E0880B04201E0E3
:109560003EE03BE001D10120E072A5841420205EA2
:10957000FCF770F802900F460398FCF77FF8284A32
:10958000284BFBF775FF05460E460198FCF762F87D
:109590002A463346FBF75EFF3B46029AFBF7B6FED0
:1095A000FCF78EF8206468460088A08313481349AE
:1095B0005030807C63316071420008460D46513066
:1095C000FBF7DCFD6079294642000C48CC30FBF704
:1095D000D5FD608BFF2801D00320207005B0F0BDC1
:1095E00000F030FFEC000020FC00002058000020BC
:1095F00000040050E1000020E2000020D81100200B
:10960000640D00200000002000D02724000100206D
:10961000180100209C140020E7030000F80000203F
:10962000F853E3A59B843E4070B586B0142168468C
:10963000FBF7BDFD01250F4EED0300222946304604
:10964000FDF7C9F9012000240190029469460095B4
:1096500003943046FDF7F6F8032001900294694622
:10966000009503943046FDF7EDF8022001F088FCE8
:1096700006B070BD000400500088704770470000BD
:10968000F8B5044600206A461080194D55222A700C
:10969000AA226A700322AA70661DEE702A7169718F
:1096A000144A49008918AC712246E81DFBF766FD93
:1096B000002007E029186A468978128889186A46C6
:1096C0001180401CB042F5DB611DA81CFCF7FEF9BF
:1096D00001466846018029190078C87168464078BB
:1096E000087221460931024800F0B8FBF8BD0000BD
:1096F000DC130020640D002010B51B4C228A01E011
:10970000891AA183A18B9142FAD2228C8BB2534346
:109710001B18E383132902D14A431018E083E08B1E
:10972000302148436421643048431049606309682C
:10973000401A4B21090140182063FBF78BFF0C4AAC
:109740000C4BFBF7FDFEFBF7BBFF0B49E0628842C9
:1097500002DD4A428018E062002801DA4018E06227
:1097600006490968486110BDDC000020980000200F
:10977000F853E3A59B843E40FF7F00009C1400202B
:10978000034A1168382389B2994301431160704735
:109790000030014010B5FDF72BF910BD10B59AB09F
:1097A00034216846FBF703FD14210DA8FBF7FFFCED
:1097B0001C2112A8FBF7FBFC1B4801680324E402F0
:1097C000A143C21489180160FDF7AAFB174801697B
:1097D000A143016106200090FF200130029001208A
:1097E0000390102004900220099040040B90000187
:1097F00000240C900A946846FDF7C0FD0F200D90E0
:1098000003200E900F941094012111940DA8FDF7E0
:109810008BFC81201290032080041890149412A8CD
:10982000FDF7D0FB1AB010BD0070004040100240A0
:1098300010480168821511430160C1680E4A114049
:10984000C16001680D4A1140016081684908490002
:10985000816001680122920491430160C168FD2288
:1098600012049143C16000210161064904488860E7
:1098700070470000001002400C40FF88F6FFF6FE23
:109880000050000800ED00E070B5026801239B075E
:10989000114C124D984203D0A04201D0A84203D1EE
:1098A0007026B2434E683243984203D0A04201D0A2
:1098B000A84204D103231B029A43CB681A43802396
:1098C0009A430B691A4302608A68C262096881621E
:1098D0000121416170BD00000008014000140140F9
:1098E00010B5CB06DB0E0121046A99408C4304625B
:1098F000016A9A401143016210BD30B58468FF25AA
:109900002D021B021343AC430B432343836030BD42
:10991000826870239A430A4307210A438260704792
:1099200030B5026A520852000262026A45688369D1
:109930007024A3439C080B68A40023430224A24381
:109940008C6845601443836149684163046230BD9B
:1099500030B5026A10239A430262036A456882693D
:1099600073242402A2430C6824021443202293434C
:109970008A68456012011A43846149688163026202
:1099800030BD30B5026AFF2301339A430262026A96
:109990004568C3697024A3439C080B68A400234353
:1099A00001246402A2438C68456024021443C3610D
:1099B0004968C163046230BD30B5026A01231B03EC
:1099C0009A430262036A4568C26973242402A2436F
:1099D0000C68240214430122520393438A684560B1
:1099E00012031A43C46149680164026230BD30B594
:1099F000036A046A6408640004628469F025AC4365
:109A0000120122430A24A3430B438261036230BD47
:109A100030B5036A1024A34303628469036A0F25E7
:109A20002D031203AC432243A024A343090119438D
:109A30008261016230BD0000F8B5102405252D07B4
:109A4000AC62AF20800001F0A2FAAC6101F01CFD15
:109A5000274C284F284E20650BE001F015FD2065AE
:109A6000FEF788FC206B411C2163142801D9234890
:109A7000C760206DB042F0D1002626632078012710
:109A8000FF03002806D001280CD0022817D0032895
:109A90002BD128E0012239462846FCF79CFFFFF72E
:109AA00075FC06E0012239462846FCF794FFFFF7D3
:109AB00065FA002239462846FCF78DFF15E0607AEA
:109AC0000122401E607239462846FCF784FFFCF7ED
:109AD000C3F9002239462846FCF77DFF607A00284A
:109AE00003D1267001E0FEF79BFF01F0B3FBF8BD48
:109AF000580000200400FA053001CADE00ED00E045
:109B000010B5818CC90707D001684A6801235B043E
:109B10009A43836A1A434A60818C890707D5016892
:109B20004A6801231B049A43C36A1A434A60818C22
:109B3000490707D501684A6801239B049A43036BD0
:109B40001A434A60818C090707D501684A680123D6
:109B5000DB039A43436B1A434A60818CC90607D5DD
:109B60000268916801231B039943836B1943916039
:109B7000818C890607D501688A6801235B039A43B3
:109B8000C36B1A438A60818C490612D503685A68F0
:109B900001210905046C8A4322435A60026C8A42FF
:109BA00007D10268516803235B059943436C19434D
:109BB0005160818C090607D501684A680123DB04DE
:109BC000806C9A4302434A6010BD0000F8B5044619
:109BD000002680300660FCF705FF05462068006817
:109BE000124F000709D501212B46002249052046C6
:109BF000009700F0ABFA00280DD1206800684007FC
:109C00000BD501212B46002289052046009700F044
:109C10009DFA002801D00320F8BD2020A067E0674E
:109C20002666603426750020F8BD0000FFFFFF01A6
:109C3000F8B5184CC826E078002829D160790028AA
:109C400026D101206071144D686B002700281ED0BA
:109C5000686BC821081A15E01048E168405C61692A
:109C600088470F480A21008848430E490880E06869
:109C7000401CE060E068C82800DBE760696BC82032
:109C8000401A761EE168814201D0002EE4DC677143
:109C9000F8BD00003C000020000002409C0C0020A9
:109CA000EC000020FE00002070B5224CE078002877
:109CB0003FD1207900283CD1012020711E4EF1694E
:109CC00000250906002933DA2156625791420AD14C
:109CD000F06940062CD5A079002829D0A5712089EB
:109CE000401C208124E0A179002903D1A0710A2021
:109CF00001F04DF900202056CC2148430F4942186D
:109D0000206912181279B262401C00222061A2560A
:109D1000CC235A43895881420ADC25612078401CB3
:109D2000207020780E2800D12570A078401CA070EB
:109D3000257170BD3C0000200038014074010020F6
:109D400010B5806A0022014640314A834A82FDF7FD
:109D500097FF10BD70B5846AA06FE56F21688968B0
:109D600000260906002906DA212804D152200653CC
:109D7000204600F06BF820688068400606D5222D4A
:109D800004D15A200653204600F047F82046803080
:109D900001681022114301602046FDF771FF70BD7C
:109DA00010B501460968806A096889061CD400223A
:109DB0005A210A5201680A68FF2301339A430A6054
:109DC00001688A68520852008A6001688A684023E4
:109DD0009A438A602021C167016E012904D101687C
:109DE0000A6810239A430A60016E012902D0FEF727
:109DF00029F910BD5821095AFDF740FF10BD10B5D3
:109E0000806A016E012902D0FEF71DF910BD5821AC
:109E1000095A4908FDF732FF10BD01680A68FF239F
:109E200021339A430A6001688A68520852008A60A6
:109E3000016E012904D101680A6810239A430A605F
:109E40002021C167002101664166704701680A68E8
:109E5000C0239A430A6020218167704770B5164C71
:109E6000E278002A0CD12279002A09D10122E2707D
:109E70000025C82903DC0222A256002A01DCE57075
:109E800070BD0123E356CC2253430C4AD150012329
:109E9000E356CC2673439B180A460146181DFBF770
:109EA0006DF96078401C607060780E2800D1657094
:109EB000A078401EA070E2E73C0000207401002062
:109EC000F8B50446016880682369E6691843636948
:109ED000002533431843724A0B68724E33400343E4
:109EE0000B602168486803231B039843E368184309
:109EF00048602168A069914201D0236A18438B68A9
:109F00000B263602B34303438B60674923686748D7
:109F10008B420CD1C0688007800F06D0012839D051
:109F2000022835D0032821D11EE001271FE0604917
:109F30008B420AD1C0680C21084027D0042829D0C0
:109F4000082825D00C2811D10EE093420ED1C1680B
:109F500003208002014019D001208002091A19D083
:109F6000091A15D0814201D1082700E010274F4976
:109F7000504840398600934232D1002F0CD0022F36
:109F80000DD0042F10D0082F7FD126E00027EEE758
:109F90000227ECE70427EAE7FDF794F906E00968F1
:109FA000C90605D4304603E0FDF7ACF9002872D0AD
:109FB000626851005118814267D81103814264D30D
:109FC000010E06025008002330185941FBF7A6F88D
:109FD00003210902411A384A55E00120C003E7E78E
:109FE0000122E369D20393422BD13B0000F0FBF93D
:109FF0000906090C4D114D4D4D274D00FDF762F935
:10A0000009E0FDF76FF906E00968C90605D4304696
:10A0100003E0FDF777F900283DD0616840004A0869
:10A020008018FBF765F880B20146244A1039914246
:10A030002BD8511C01400007400F084329E010466F
:10A04000EBE73B0000F0CFF90906090C21122121B2
:10A0500021232100FDF736F90AE0FDF743F907E077
:10A060000968C90606D4304604E00EE0FDF74AF957
:10A07000002810D061684A081018FBF739F880B240
:10A0800001460E4A1039914203D9012503E01046DA
:10A09000F0E72168C86000206066A0662846F8BD29
:10A0A00000480040F369FFEF0038014040100240D3
:10A0B0000044004000093D00FFFC0F00EFFF0000DE
:10A0C000F8B50446416540300026274602838037B4
:10A0D0003E602220E0672546206F603500281CD0B6
:10A0E0001749C162216F17480863216F16484863FA
:10A0F000206F8663236F606D9C461346216802467D
:10A1000060462431FCF7C6FA002806D010203860DB
:10A110002E752020A0670120F8BD2E7520680168EB
:10A12000FF2201321143016020688168012211433E
:10A130008160206881684022114381600020F8BD61
:10A14000A19D0008FF9D0008559D0008FFB581B046
:10A1500005460F46044660350A9E39E0701C37D02C
:10A16000FCF740FC0499401AB04222D8002E20D0BF
:10A170002068016849072BD5C069C043000527D472
:10A1800001202168C002086220680168FF22A13214
:10A19000914301602068816849084900816020205E
:10A1A000A067E0678034206000202875032005B098
:10A1B000F0BD20680168FF22A13291430160206850
:10A1C00081684908490081602020A067E067EBE7CB
:10A1D0002068C1693846884305D000210398814230
:10A1E000BCD00020E3E70121F8E7000010B50449E6
:10A1F0001020096808620248FDF744FD10BD000008
:10A200006415002001B501231A4669460248FDF78E
:10A210001BFF0248C06908BD6415002000380140DA
:10A2200001490D20887070473C00002010B5074898
:10A230000A22018A51434184FEF7B0FAFEF7C8FBB7
:10A24000C82203490348FDF7CDFE10BDDC00002005
:10A250009C0C002064150020F8B53E4C00232178AA
:10A260003D4A1D46082910D0072947D0062950D05D
:10A27000052952D0042953D0032954D0002956D09F
:10A28000012958D002295AD05BE0A17800264A1F44
:10A2900004E0314FBF5DFB189BB2761C9642F8DBA1
:10A2A000667927799A195118E3786278C91889185C
:10A2B000C9194018C0430006000E1AD1012E14D04F
:10A2C000022E16D125482449C018FAF757FF01F08D
:10A2D000DBFB642000F054FEBFF34F8F2149204880
:10A2E000C860BFF34F8F00BFFDE759081046FFF766
:10A2F000C7F92570E570A570A571F8BDA179505416
:10A30000491CC8B2A071A178491F8842F5D1082024
:10A3100001E0607007202070F8BDE0700620FAE7C9
:10A3200060710520F7E7A070E5700420F3E7552879
:10A3300007D10120EFE7AA2803D10220EBE7032889
:10A3400003D02570E570A570F8BD03202070207142
:10A35000F8BD0000D300002078130020640D002019
:10A360000400FA0500ED00E00FB410B503A9044B9A
:10A37000044A029800F004FA10BC08BC04B0184764
:10A38000BDB70008340100202021020C01D01021AB
:10A390001046020A01D010460839020901D01046C1
:10A3A000091F820801D01046891E420801D0881E6C
:10A3B0007047081A7047F8B5040C8BB2264682B273
:10A3C0005E430D0C1046370C5843360480190021AB
:10A3D000794116466E43370C36048019794126467A
:10A3E0006E438919F8BD30B47446641E2578641C28
:10A3F000AB4200D21D46635D5B00E31830BC1847DA
:10A400008307FF22DB0E9A408907090E9940002836
:10A4100008DB830809489B001B1818689043084311
:10A42000186070470007000F0838830804489B0035
:10A430001B18D86990430843D861704700E400E0D6
:10A4400000ED00E0BFF34F8F04490348C860BFF33D
:10A450004F8F00BFFDE700000400FA0500ED00E0AB
:10A4600002E008C8121F08C1002AFAD170477047DD
:10A47000002001E001C1121F002AFBD1704708B57E
:10A480000021684601706B46012202212C2001F058
:10A4900035F90221684601706B4601222C2001F03B
:10A4A0002DF908BD38B504466D20694608706B4625
:10A4B000012207492E2001F021F90649002C01D084
:10A4C000054A00E0054A2E2001F0FEF838BD0000E4
:10A4D0000608000006180000070600000716000026
:10A4E00038B504466B4602220021362000F0D2FF28
:10A4F000B3212300FFF777FF0E0F08153A3A3A3AD7
:10A500001C273A3A2F34483A0021684601704078B7
:10A510004108490014E06946087880088000401C22
:10A5200004E06946087880088000801C08701DE0FF
:10A53000684602780A404832027041788020014320
:10A540006846417012E0684602780A40027040781E
:10A550004106490EF4E7694648780221084303E0C2
:10A5600069464878FD210840694648706B460122DB
:10A570000021362001F0C2F8012200AB114636203E
:10A58000013301F0BBF838BD69460878CF21084097
:10A5900069462030CAE708B50321684641700121A9
:10A5A00001706B4602220021362001F0A7F801223B
:10A5B000D20306212D2001F087F8012000F0E0FCF5
:10A5C0000120FFF78DFF08BD08B5020A69464A70F1
:10A5D00008706B46022204212D2001F08FF8032021
:10A5E000694608706B46012206212D2001F086F88D
:10A5F0000020694608706B46012206212D2001F0DB
:10A600007DF80A212D2000F02BFF08BDF0B51FB406
:10A6100086B00998089A030D0021024314D05148CE
:10A62000514A1818504305141198012810981AD04F
:10A63000281A401C00264D4F4D4900960191049068
:10A64000002812DA444211E01198012449A301289C
:10A6500001D11098C1430698119A84600360C260CA
:10A6600041600BB0F0BD4042E4E704462105002004
:10A670003F4A001C51410391029012E0E00707D0CD
:10A6800032463B4601990098FAF7F2FE019100909C
:10A6900032463B4610461946FAF7EAFE06460F4692
:10A6A0006410002CEAD10498039B0028029A0999AF
:10A6B000089806DAFAF7DCFE019B009AFAF7D8FE52
:10A6C00005E0FAF73DFF019B009AFAF739FF0446CF
:10A6D0000E460022284BFBF749F803D80020C04360
:10A6E000014607E00022254B20463146FAF70EFED0
:10A6F000FBF74AF9102409E0002C0ADB0A220023A8
:10A70000FAF70CFD079B30321A55641E02460A43C5
:10A71000F2D11122641C079B121B1C19119B012BE7
:10A7200003D0012308430ED10AE0084304D01120CE
:10A7300010900020119077E71098151A6D1E0BE00D
:10A740001098824202DD00236D1C03E0824201DA90
:10A7500000236D1E002BEED0069811998260C16017
:10A7600030C07EE701FCFFFF104D000000001440E8
:10A770000000F03F300000000000F0430000E03F28
:10A78000FFB597B00646002518E2252877D10024AA
:10A790002746FD49049400E00443761C32780120EA
:10A7A000203A90400842F7D130782A280ED0022271
:10A7B000307801463039092916D804990A235943BB
:10A7C000303940181443761C0490F1E7189802C8F9
:10A7D00004911890002904DA012040030443484200
:10A7E000049002200443761C30782E2814D10420D3
:10A7F00004437078761C2A2809D11898761C80C8E2
:10A80000189009E00A214F43303FC719761C307871
:10A81000014630390929F5D930786C2810D006DC8A
:10A820004C281AD068280ED06A2817D104E0742862
:10A8300013D07A2812D110E00120400504430CE027
:10A840000121090501E0032109050C4371788142CA
:10A8500003D1012000052418761C761C3078119055
:10A8600066280BD013DC58287DD009DC00287BD06B
:10A870004528F6D04628F4D047281AD1A5E118E09B
:10A88000632835D0642870D0652812D19DE17028E6
:10A890006CD008DC6728F1D069287BD06E280DD0F9
:10A8A0006F2806D1BAE073282ED0752871D0782889
:10A8B00059D01A9A199990476D1C7EE16002400F99
:10A8C000022809D003280DD00428189801680DD05B
:10A8D0000D60001D189070E11898EA1701680D606E
:10A8E0004A60F6E7189801680D80F2E70D70F0E70E
:10A8F00018986A4601781172001D18900020507255
:10A9000002A80090012005E0189802C818900020C5
:10A910000091C04361070DD5002101E00199491C58
:10A920000191B94212DA8142F8DB009A515C0029A8
:10A93000F4D10BE0002101E00199491C0191814211
:10A94000FADB019A0099895C0029F5D101990498F4
:10A950001A9B471A21463846199A00F097FA01992E
:10A96000401945180BE04FE02CE113E04EE0009851
:10A9700000990078491C00911A9A199990470198FA
:10A98000401E0190401CF2D1214638461A9B199A6C
:10A9900010E137E00A200021009001916002410F90
:10A9A000022907D0189A01CA1892C217944603299F
:10A9B00008D00AE01898C01DC108C90005C918913F
:10A9C000944607E000B2C2179446042902D140B26F
:10A9D000C1178C4600226146944506DA0A460021DA
:10A9E000404291418C462D2102E0210504D52B21C6
:10A9F0006A461173012103E0E10701D02021F7E746
:10AA0000029155E00A200AE0102008E01020009092
:10AA10000021042004430191082703E008200021BD
:10AA2000019100906002410F022907D0189A01CAD3
:10AA3000189200229446032908D008E01898C01DF7
:10AA4000C108C90005C91891944603E080B20429E1
:10AA500000D1C0B200210291210729D51199702996
:10AA600006D0009A1021019B4A401A4305D00EE0FF
:10AA700040216A461173012108E06146014306D076
:10AA800030216A4611731199517302210291009A83
:10AA90000821019B4A401A430AD16146014301D172
:10AAA000610705D530216A46117301217F1E02918D
:10AAB0001199582904D035A10E910DA90D910DE0E1
:10AAC00037A1F9E76146019B009AFAF727FB0E9B35
:10AAD0008C469B5C0D9A521E0D9213706146014389
:10AAE000F0D10D9805A9081A20300190600703D510
:10AAF00001200004844300E001270198874201DD22
:10AB0000381A00E0002001990090411802980918B5
:10AB10000498401A0490E00306D421461A9B199A1F
:10AB2000049800F0B3F94519002706E003A81A9A23
:10AB3000C05D199990476D1C7F1C02988742F5DB18
:10AB4000E0030CD521461A9B199A049800F09EF94F
:10AB5000451904E01A9A3020199990476D1C009904
:10AB6000481E00900029F5DC08E00D980D9900784A
:10AB7000491C0D911A9A199990476D1C0199481E0C
:10AB800001900029F1DC63E1092801003031323302
:10AB90003435363738396162636465660000000019
:10ABA0003031323334353637383941424344454603
:10ABB0000000000000F05AF94519761C3078002892
:10ABC00000D0E2E528461BB0F0BD600700D40627A0
:10ABD0001898C01DC108C90048680A680831C30F29
:10ABE000DB071891190001D09CA108E0210501D5CF
:10ABF0009BA104E0E10701D09AA100E09AA14300E3
:10AC000011985B08109165280CD006DC452809D006
:10AC100046281DD0472841D141E0662818D0672832
:10AC20003CD13CE00021112F01DB112000E0781C19
:10AC30000191009008A911A8FFF7E8FC139905916C
:10AC40000021119A15927F1C12980197009150E0F3
:10AC50000120C00703900120019008A9009711A8C6
:10AC6000FFF7D4FC139A149905920022119B0092CD
:10AC700012981593059A0192002901D0104602E01E
:10AC8000791C40180190381A01D5019804E040421F
:10AC9000401E0090781C0190C01B029043E0012FE1
:10ACA00000DA01270021112F01DD112000E03846D4
:10ACB0000191009008A911A8FFF7A8FC139905912C
:10ACC000119A0021129815920091019721070CD436
:10ACD0000599B94201DB019900E00191012904DDE8
:10ACE000159A491E515C302906D0B84201DA011D7F
:10ACF00005DA0121029115E00199491EEDE70028CE
:10AD000005DC0099411800910199091A03E0019AA4
:10AD1000411C914200DD01910099401A401C0290B3
:10AD20000120C0070390200706D4029901988142B0
:10AD300002DB0020C043029000206946C87707AFBD
:10AD4000012103980337C907884224D002201190BB
:10AD50002B201290039800280CDA404203902D20FB
:10AD6000129007E00A210398FAF7C2F930317F1EEA
:10AD7000039039701199481E11900029F2DC039854
:10AD80000028EFD1791E12980870307820210840F1
:10AD90004530BF1E387006A8C01BC01D0390109818
:10ADA0000078002800D00120019941180298C017AE
:10ADB0000918039809180498401A401E0490E003EB
:10ADC00006D421461A9B199A049800F05FF8451999
:10ADD00010980078002803D01A9A199990476D1C92
:10ADE000E00324D521461A9B199A049800F04EF8E6
:10ADF00045191CE00098002807DB00990598884257
:10AE000003DD1598405C199901E0199930201A9AD0
:10AE1000904700986D1C401C00900298401E0290C4
:10AE2000002804D11A9A2E20199990476D1C019977
:10AE3000481E01900029DDDC05E038781A9A7F1C55
:10AE4000199990476D1C0399481E03900029F4DC62
:10AE500021461A9B199A0498ACE600002D000000C8
:10AE60002B0000002000000000000000F8B50446A0
:10AE700000251E461746880404D405E039462020E4
:10AE8000B0476D1C641EF9D52846F8BDFFB50446D1
:10AE9000002581B01E46C80301D5302700E02027D9
:10AEA000880404D505E038460399B0476D1C641E3C
:10AEB000F9D5284605B0F0BDF8B54A002B4B520D28
:10AEC000D6182B4A0C460546142E2BDA002E12DA21
:10AED000284BFAF71BFA00221346FAF747FC40D238
:10AEE000002C03DA0124E40700253AE02046284339
:10AEF00037D0214C14E0214F0B46F7403B402B4309
:10AF000031D01C4BFAF702FA00221346FAF72EFC56
:10AF100027D2002C03DD01200005F0400419BC43BA
:10AF200000251EE0332E1EDC33460027143BFF4372
:10AF3000DF40384217D00F4BFAF792FA002213463F
:10AF4000FAF714FC0DD2002C0ADD142E0CD034209C
:10AF5000811B012088404019A84200D2641C05468C
:10AF6000BD4321462846F8BD641CF9E701FCFFFFFC
:10AF70009C7500883CE4377E0000F03FFFFF0F0027
:10AF80007D2110B5C900484300F001F810BD002133
:10AF900040E000BF00BF00BF00BF00BF00BF00BF58
:10AFA00000BF00BF00BF00BF00BF00BF00BF00BFA9
:10AFB00000BF00BF00BF00BF00BF00BF00BF00BF99
:10AFC00000BF00BF00BF00BF00BF00BF00BF00BF89
:10AFD00000BF00BF00BF00BF00BF00BF00BF00BF79
:10AFE00000BF00BF00BF00BF00BF00BF00BF00BF69
:10AFF00000BF00BF00BF00BF00BF00BF00BF00BF59
:10B0000000BF00BF00BF00BF00BF00BF00BF00BF48
:10B0100000BF491C8142BCD370470000FEB5044606
:10B020000020019000906079734940000E5A6178C9
:10B030002578491E7148CFB20163042D77D0072DC2
:10B0400075D000210291217801736C49E3790122C6
:10B0500092058969002B6CD0914381616748217A00
:10B060004173217A82698907890B0A438261002131
:10B07000042000F034FB324661492E2000F024FB0E
:10B080003846FFF70FFA5F4E0522705D81004018C9
:10B090005D49431807212B2000F030FB5B490298E3
:10B0A00001220B180B21282000F028FB705D584965
:10B0B00080000A580C21282000F011FBE079554946
:10B0C00080004018A1794900425A0221272000F04F
:10B0D000FBFA51487E00825B0421272000F0F4FA3D
:10B0E000E079002829D0A07804282CD028206946AF
:10B0F000087220220621272000F0E6FA02AB012286
:10B100002621272000F0FAFA444938014018E17856
:10B11000890042580821272000F0E1FAA17A601C3A
:10B12000627A0902114313D016E000E001E0012128
:10B1300088E71143F608816190E764220621272001
:10B1400000F0C2FAE0E71020694608720246D1E733
:10B1500033490172090A4172417A007A0A020243B4
:10B160002021272000F0B0FA2E4F0C2123203A682E
:10B1700000F0B5FAF01982880421232000F0A4FA27
:10B18000A07900280BD0E07927490122431800213B
:10B19000212000F0B3FA03200190012000902A073B
:10B1A000120F10010243607800218007000B024358
:10B1B0000198000502430098400402432079C0062C
:10B1C000400902436079C00602431F2000F087FA5D
:10B1D000A07861780123084302040848DB03026178
:10B1E000E179490319430A4302610021082000F074
:10B1F00076FA0020FEBD000054BB00083801002094
:10B2000004280000FCBA00080C0000202A000020DE
:10B2100004BB000824BB000830BB000834BB000896
:10B22000411000001CBB00082C00002038B50C4663
:10B2300007498A8B002102432C2000F045FA68461A
:10B2400004706B46012206212C2000F057FA38BD0D
:10B250003801002010B5FFF712F910BD10B50446F3
:10B260000421362000F0FCF80121C902002C01D095
:10B27000084300E0884302460421362000F02FFAFC
:10B2800010BD000038B540206946087000210E202E
:10B2900000F0E6F80446002211460E2000F01FFAE6
:10B2A0006B46012200210D2000F028FA074A0021F8
:10B2B0000F2000F014FA00F0EDF9224600210E20D4
:10B2C00000F00DFA02480021017338BDF8FF272471
:10B2D00058010020FEB50546042069460870514C0F
:10B2E0000020607521462031206348710873A083D7
:10B2F0006063A06300F0C8F84B4E206002E000F0ED
:10B30000C3F82060B042FAD10020FFF7E9F800F05E
:10B31000BBF8464E20603078242801D9243806E056
:10B320000621F9F7E5FE0622101A4001084302063D
:10B3300001040A4301020A430243B2607060002123
:10B340001E2000F0CCF900F09FF820606B4601222F
:10B350000021242000F0D2F91E20FFF735F986B233
:10B36000300AA0730420FFF72FF9074600F08CF88D
:10B3700020603806000E0DD002206946087101AB2E
:10B38000012212212D2000F0B9F9A08B012109031F
:10B390000843A08300F078F820600620FFF714F936
:10B3A00060600720FFF710F9A060F006C00E20755E
:10B3B00001D110202075C0B200F0DCF9E80707D0F9
:10B3C000FFF7E9F8A08B0121C9020843A0830AE036
:10B3D0000521362000F02EF81549084002460521C7
:10B3E000362000F071F90120FFF77AF800210420DF
:10B3F00000F036F8A0610021262000F031F8152178
:10B400008903084302460021262000F068F9002243
:10B410002621362000F058F900F036F82060002090
:10B42000FEBD0000380100203001CADE000000200F
:10B43000FFFD000038B5094C89B280B26B4602228C
:10B4400000F028F8002806D16846407801026846D6
:10B450000078081884B2204638BD0000FFFF0000C5
:10B4600038B50024E44389B280B26B46042200F070
:10B4700011F8002806D103216846435C2202D41843
:10B48000491EFAD5204638BD10B500210846FFF701
:10B49000E7FF10BD38B5002909D0402420436C4691
:10B4A0002070C8B27F2906D8607002200AE0694681
:10B4B0000870012006E0802420436C466070C809B3
:10B4C000A0700320694600F0B9FA38BD10B51446E3
:10B4D00003460A4621461120FFF7DCFF10BD10B5D8
:10B4E0000346052200211520FFF7D4FF10BD10B53B
:10B4F0000346052200211720FFF7CCFF10BD38B509
:10B50000054600206946087000F0C4F8FF240134A5
:10B510002246002D01D00322120200210D2000F04E
:10B52000D3F8002D13D06B46012203210F20FFF723
:10B53000B1FF68460078000709D5FFF7A3FE224651
:10B5400000210D2000F0C0F80020C04338BD0020CD
:10B5500038BD10B5024601210A2000F0C0F810BD28
:10B5600010B5044600211A20FFF77AFF000D2203D0
:10B570000005120B024300211A2000F0B0F810BDA4
:10B5800010B5024602492E2000F09EF810BD0000C2
:10B5900004180000F8B505466B460122032104207B
:10B5A000FFF778FF0126114C3607002D0DD02A46F3
:10B5B00000210C2000F088F8694608781021084323
:10B5C00069460870A069304307E069460878EF21B2
:10B5D000084069460870A069B0430B46A06101228B
:10B5E0000321042000F08AF8F8BD00003801002093
:10B5F00010B502460021182000F066F810BD0000CA
:10B60000F8B50746002568460570B807204C2E4659
:10B6100000280ADA8020694608706B460122002162
:10B620000D2000F06BF801202073F80769460878B8
:10B6300021D006210843694608706B46012200218B
:10B640000D2000F05BF803210F20FFF7F3FE8121AE
:10B65000C900084219D04020694608706B46012293
:10B6600000210D2000F04AF80020FFF7F7FD00252B
:10B670002673ED4309E002210843694608706B46D2
:10B68000012200210D2000F039F82846F8BD000005
:10B69000580100201CB56B46012203210F20FFF743
:10B6A000F9FE684600784022C1091040C9014000F7
:10B6B000814208D0012069460871024601AB03218E
:10B6C0000D2000F01BF81CBD08B56B461A70120A5D
:10B6D0005A7089B280B2022200F010F808BD38B565
:10B6E00000236C46E254120A5B1C042BFADB89B27D
:10B6F00080B22346042200F001F838BD38B580241A
:10B70000002909D0C02528436D462870C8B27F297A
:10B7100007D86870022009E02043694608700120BC
:10B7200004E020436870C809A8700320694600F04F
:10B73000C1F938BD10B51446012312189B029A4274
:10B7400002D90020C04310BD0B46821E21460920AD
:10B75000FFF7D4FF002010BD10B5054A8905126916
:10B7600001430A4300210820FFF7B9FF002010BD64
:10B770003801002038B504466B4601220E212B20EB
:10B78000FFF788FE68460078E10640094001C90ECF
:10B790000143684601706B4601220E212B20FFF702
:10B7A000ADFF38BD10B5002142541C06120A2243D9
:10B7B0001B0A491C0429F7DB10BD000013B5012347
:10B7C0001A4669460248FCF73FFC00981CBD000081
:10B7D000641500207CB5002425466846FFF77FFEEF
:10B7E00004206946220E2D02154322020C5C1443EC
:10B7F000401EF7D5204629467CBD7CB50024254651
:10B800006846FFF774FE04206946220E2D02154398
:10B8100022020C5C1443401EF7D5204629467CBD0D
:10B82000FBF7EEF8FDF7BAFFFCF7CCFF41494248C1
:10B83000002522C005608561C56140490562C1607F
:10B840000838FBF779FAFCF7A9FFFDF7C1F8FDF717
:10B850005DF8FCF76FFF052601223607D10330465D
:10B86000FBF7B9F8FDF718FDFCF758FEFAF78EF96B
:10B87000FAF75CF9FCF75AFC0721B015FFF7D6FC84
:10B88000FFF7E8FC2E4C0A21208A012248436084FD
:10B8900011033046FBF79FF82748C8222949C830D2
:10B8A000FCF7A0FB284F294E207900283FD0607874
:10B8B00000283CD0FDF772FF2571FAF753FB20708A
:10B8C0000F280AD9012211033046FBF784F8FEF74E
:10B8D000B3F800220121090309E001225103304697
:10B8E000FBF779F8FEF7A8F800220121490330465A
:10B8F000FBF771F8FCF73EFD608C002801D0401E7C
:10B9000060841348618C00780843CDD138780028D2
:10B9100001D00328C8D10121C9023046FBF74EF8F7
:10B920000028C1D101210846FBF71AFBBCE7FCF750
:10B9300021FDB9E7007C00409C140020FFFF0000BF
:10B94000DC0000209C0C0020690000200004005056
:10B950004200002010B586B01748FBF770F914219B
:10B960006846F9F724FC1548009003200190002058
:10B970000290052069460007FAF764FF69461048FF
:10B98000FAF760FF69460F48FAF75CFF01210846A5
:10B99000FBF7E6FAFF2401342046FBF7B9FA0A491F
:10B9A00008680422104308602046FBF7C1FAFBF741
:10B9B000C7FA06B010BD00009C140020FFFF000075
:10B9C00000040050000800500070004010B5012233
:10B9D000920217491748FAF765F91548164902887F
:10B9E0008A4223D00180FF2101318180FF21F5317E
:10B9F000C1800A21018100211E224181D24382811E
:10BA00000122C28181831E23C386022303877823F8
:10BA100043878287C28702464032118451849184D1
:10BA2000C18391801421818200F02EF810BD0000A6
:10BA3000640D002000FC0008AA550000F0B58C46FB
:10BA400000251026052109078E620E4C08E0674686
:10BA50007F5DE760A768FF07FCD0E7681F706D1C7B
:10BA60008542F4DB0020074606E0E760A568ED07A5
:10BA7000FCD0E5681D54401C9042F6D38E61002036
:10BA8000F0BD00000030014070B572B60124074DD2
:10BA9000A40221462846FAF7EBF8002804D02246F3
:10BAA00003492846FAF788F962B670BD00FC000821
:10BAB000640D0020F0B50025102605279C463F07A1
:10BAC0000B46BE620C4C06E0595DE160A168C907F7
:10BAD000FCD0E1686D1C8542F6DB002007E0614682
:10BAE000095CE160A168C907FCD0E168401C904294
:10BAF000F5D3BE610020F0BD00300140000001021E
:10BB000003040005405C0000A05C0400C06C080059
:10BB1000805C0400E03F1E00E07D1E0007A90225B6
:10BB200070889B880A0016000100060001000200D0
:10BB300087008D002D001A3152001A339A001A35F1
:10BB40001D011A376B003B31BE003B335E013B35B4
:10BB500096023B37000099599959EB518F421E4587
:10BB6000142E0080EB51F5283333E13A703DE13A71
:10BB7000C235852BC2353333C235C235AE47E13AC3
:10BB80005138A330513800000000000000000102CD
:10BB9000030406070809030406080C1018203000E7
:10BBA0000000000102030400C8BB000800000020E0
:10BBB00038010000EC59000808BC000838010020DA
:10BBC0005819000070A40008C1130704380D091E9D
:10BBD000080540082609104008560A131D043B08B2
:10BBE000BE0516D8BC40100852010334C842035A9F
:10BBF0005C121B0202BD14090102628149A80146C0
:08BC0000294C920452200000BF
:04000005080050C1DE
:00000001FF
